:100000000C9400070C9444070C9444070C94440788
:100010000C9444070C9444070C9444070C94440734
:100020000C9444070C9444070C9458120C942A1313
:100030000C9444070C9444070C9444070C94440714
:100040000C9444070C94022C0C9444070C94440721
:100050000C9444070C94FA210C9444070C94440724
:100060000C9444070C9444070C9444070C944407E4
:100070000C9444070C9444070C9444070C944407D4
:100080000C9444070C9444070C9444070C944407C4
:100090000C9444070C9444070C9444070C944407B4
:1000A0000C9444070C9444070C9444079713B91319
:1000B000A714B913A714FE132114A71476148914D6
:1000C000D017D017FF17FF17431881189B1A9B1AD8
:1000D0009A189B1A9B199B196F1A9B1A9B1A861ABE
:1000E0000000F0A12E002B002971E10035810000F5
:1000F0001E00140004001D71E20027021F001A00F8
:1001000016001B00E104E3002000080007000600C1
:1001100050002C0021001500090019004F00260294
:10012000220017000A000500000065743400C100B9
:100130000000007F0000E3003400C10000000077F1
:100140000000290023001C000B0011000000297191
:10015000240018000D00100052002F0225000C0092
:100160000E00360051002800260012000F00370054
:100170002F00E7002700130033823871300030026F
:100180002A002D003100E5000154000001000100AB
:1001900001000100010000003A001E0220022202BC
:1001A000010001003B001F022102230201000100A7
:1001B0003C002F0226022F00010001003D0030020A
:1001C00027023000010001003E00310235003502F7
:1001D000000001000100010000000100000001001A
:1001E0000100010000000100000001003F0052007A
:1001F00051002402000001004000240021001E00E4
:10020000010001004100250022001F00370001000D
:1002100042002600230020002700010043002502A1
:100220002E0231002E0001004400450001000100B3
:1002300001000000010001000100010001000000B8
:1002400001000100010001000100010001000100A6
:10025000F2000100010001000100F000F1000100C6
:10026000F400010001000100F3000100F5000100AD
:100270000100010001000100000001000100010077
:100280000000010000000100010001000000010069
:100290000000010001000100010001000000010058
:1002A0000100010001000100A9000100010001009E
:1002B0000100AC00AA00B600010001000100AB0083
:1002C000A80001000100010001000100010001007F
:1002D00001000100AE000100010000000A0025300D
:1002E000313662003A200025303258000A722F63FE
:1002F0002030313233343536373839414243444582
:10030000460A000A002530325800626F756E636538
:10031000213A20006C6566742073696465206174FD
:100320007461636865640A006C656674207369644F
:1003300065206E6F7420726573706F6E64696E678E
:100340000A00747279696E6720746F207265736534
:1003500074206D637032333031380A000A444542EC
:1003600055473A20656E61626C65642E0A005B73C6
:100370005D004B6579626F617264207374617274A1
:100380002E0A005B575D005B535D005B525D005BB6
:10039000445D005B435D0016034500720067006F1B
:1003A0000044006F007800200045005A000000164D
:1003B000034500720067006F0044006F0078002062
:1003C0000045005A0000000403090409028D0005DD
:1003D0000100A0FA09040000010301010009211134
:1003E000010001223F000705810308000A090401FA
:1003F000000103010200092111010001224D000743
:1004000005820308000A0904020001030000000934
:1004100021110100012236000705830308000A09A3
:100420000403000203000000092111010001222041
:1004300000070584032000010705040320000109CB
:100440000404000103000000092111010001223908
:1004500000070585031000011201100100000008CB
:10046000EDFE071301000102000105010906A101CB
:10047000050719E029E71500250195087501810296
:100480000508190129059505750191029501750366
:100490009101050719002977150025019578750147
:1004A0008102C00631FF0974A1010975150025FFFD
:1004B0009520750881020976150025FF952075089D
:1004C0009102C005010980A101850216010026B72D
:1004D000001A01002AB700751095018100C0050CB3
:1004E0000901A1018503160100269C021A01002AB8
:1004F0009C02751095018100C005010902A1010946
:1005000001A10005091901290515002501950575A9
:100510000181029501750381010501093009311539
:1005200081257F95027508810609381581257F95FB
:100530000175088106050C0A38021581257F950191
:1005400075088106C0C005010906A101050719E06B
:1005500029E71500250195087501810295017508A7
:10056000810105081901290595057501910295017B
:10057000750391010507190029FF150025FF950650
:1005800075088100C00A002530325820006B65795B
:10059000626F6172645F7265706F72743A20000AF4
:1005A0000025303258006B6579626F6172645F7349
:1005B00065745F6C65643A200064656C5F6B657997
:1005C0005F6269743A2063616E27742064656C3AD7
:1005D00020253032580A006164645F6B65795F6280
:1005E00069743A2063616E2774206164643A20253F
:1005F0003032580A00646F6E652E0A00626F6F67B2
:100600006D61676963207363616E3A202E2E2E2020
:1006100000290A002575002F002575005D2800259A
:10062000640020002564002000256400200025646B
:10063000007C0025303258006D6F7573656B6579ED
:10064000205B62746E7C782079207620685D287249
:1006500065702F61636C293A205B006D6B5F776872
:1006600065656C5F74696D655F746F5F6D6178203F
:100670003D2025640A006D6B5F776865656C5F6D72
:1006800061785F7370656564203D2025640A006DA4
:100690006B5F74696D655F746F5F6D6178203D207D
:1006A00025640A006D6B5F6D61785F7370656564CA
:1006B000203D2025640A006D6B5F696E746572765B
:1006C000616C203D2025640A006D6B5F64656C6180
:1006D00079203D2025640A006D6B5F776865656C45
:1006E0005F74696D655F746F5F6D6178203D202573
:1006F000640A006D6B5F776865656C5F6D61785F3C
:100700007370656564203D2025640A006D6B5F741D
:10071000696D655F746F5F6D6178203D2025640AA7
:10072000006D6B5F6D61785F7370656564203D205F
:1007300025640A006D6B5F696E74657276616C206A
:100740003D2025640A006D6B5F64656C6179203D16
:100750002025640A000A00257500363A207768656E
:10076000656C5F74696D655F746F5F6D61783A2069
:10077000000A00257500353A20776865656C5F6D65
:1007800061785F73706565643A20000A0025750022
:10079000343A2074696D655F746F5F6D61783A20DB
:1007A000000A00257500333A206D61785F7370652B
:1007B00065643A20000A00257500323A20696E749B
:1007C000657276616C286D73293A20000A002575E0
:1007D00000313A2064656C6179282A31306D7329C3
:1007E0003A20000A092D2056616C756573202D0A88
:1007F000004D3E004D25643E20003F00736574208F
:1008000064656661756C740A00433E200077686514
:1008100072652064656C74613A20637572736F72DF
:100820003D25642C20776865656C3D25640A536519
:100830006520687474703A2F2F656E2E77696B6926
:1008400070656469612E6F72672F77696B692F4DD0
:100850006F7573655F6B6579730A000A092D204D0A
:100860006F7573656B6579202D0A4553432F713A77
:1008700009717569740A313A0964656C6179282ACD
:1008800031306D73290A323A09696E746572766186
:100890006C286D73290A333A096D61785F7370654E
:1008A00065640A343A0974696D655F746F5F6D61E0
:1008B000780A353A09776865656C5F6D61785F73B2
:1008C000706565640A363A09776865656C5F7469B6
:1008D0006D655F746F5F6D61780A0A703A097072B6
:1008E000696E742076616C7565730A643A09736584
:1008F000742064656661756C74730A75703A092BAF
:10090000310A646F776E3A092D310A706775703A53
:10091000092B31300A7067646F776E3A092D3130D8
:100920000A0A7370656564203D2064656C746120FB
:100930002A206D61785F7370656564202A202872B3
:100940006570656174202F2074696D655F746F5FD9
:100950006D6178290A003F004D3E2000433E200093
:100960004C25640A000A092D20436F6E736F6C6575
:10097000202D0A4553432F713A09717569740A6D28
:100980003A096D6F7573656B65790A000A092D2048
:100990004D61676963202D0A643A09646562756771
:1009A0000A783A096465627567206D6174726978C6
:1009B0000A6B3A096465627567206B6579626F61DD
:1009C00072640A6D3A096465627567206D6F7573AC
:1009D000650A763A0976657273696F6E0A733A0929
:1009E0007374617475730A633A09636F6E736F6C25
:1009F00065206D6F64650A302D343A096C61796544
:100A000072302D34284631302D4634290A50617514
:100A1000733A09626F6F746C6F616465720A653A4C
:100A200009656570726F6D0A6E3A094E4B524F0A36
:100A30007A3A09736C656570204C4544207465737F
:100A4000740A000A002575002E6E6B726F3A200042
:100A50000A002575002E737761705F6261636B73A6
:100A60006C6173685F6261636B73706163653A2088
:100A7000000A002575002E737761705F67726176DA
:100A8000655F6573633A20000A002575002E6E6F5E
:100A90005F6775693A20000A002575002E7377613B
:100AA000705F72616C745F726775693A20000A004A
:100AB0002575002E737761705F6C616C745F6C6775
:100AC00075693A20000A002575002E636170736C09
:100AD0006F636B5F746F5F636F6E74726F6C3A20DD
:100AE000000A002575002E737761705F636F6E7466
:100AF000726F6C5F636170736C6F636B3A20000A96
:100B00000025303258006B65796D61705F636F6EE0
:100B10006669672E7261773A20000A002575002EFB
:100B20006D6F7573653A20000A002575002E6B65A0
:100B300079626F6172643A20000A002575002E6D9B
:100B400061747269783A20000A002575002E656E7E
:100B500061626C653A20000A0025303258006465F5
:100B60006275675F636F6E6669672E7261773A20A0
:100B7000000A0025750064656661756C745F6C61C0
:100B80007965723A20003F004E4B524F3A206F6613
:100B9000660A004E4B524F3A206F6E0A0074696D20
:100BA00065725F636F756E743A202530346C580A35
:100BB000006B6579626F6172645F6E6B726F3A2071
:100BC00025580A006B6579626F6172645F69646CB5
:100BD000653A2025580A006B6579626F6172645F1F
:100BE00070726F746F636F6C3A2025580A00686FDB
:100BF00073745F6B6579626F6172645F6C65647357
:100C000028293A2025580A000A092D2053746174B6
:100C10007573202D0A004743433A20342E392E3372
:100C2000204156522D4C4942433A20312E382E3124
:100C3000204156525F415243483A20617672350A4C
:100C4000004F5054494F4E533A204C554641204294
:100C50004F4F544D41474943204D4F5553454B4508
:100C6000592045585452414B455920434F4E534FFC
:100C70004C4520434F4D4D414E44204E4B524F204A
:100C80003531320A004255494C443A2030663263CD
:100C9000373733202831313A30393A3531204A61FB
:100CA0006E2020352032303136290A005649443A28
:100CB00020307846454544284572676F446F782058
:100CC000455A29205049443A20307831333037286A
:100CD0004572676F446F7820455A29205645523A2D
:100CE000203078303030310A00444553433A207484
:100CF0002E6D2E6B2E206B6579626F61726420669B
:100D000069726D7761726520666F72204572676FD8
:100D1000646F780A000A092D2056657273696F6E38
:100D2000202D0A000A6D6F7573653A206F66660A9A
:100D3000000A6D6F7573653A206F6E0A000A6B6565
:100D400079626F6172643A206F66660A000A6B65A9
:100D500079626F6172643A206F6E0A000A6D617485
:100D60007269783A206F66660A000A6D617472696A
:100D7000783A206F6E0A000A64656275673A206FE0
:100D80006E0A000A64656275673A206F66660A003B
:100D90000A0A626F6F746C6F616465722E2E2E206A
:100DA00000433E20006565636F6E6669673A0A001E
:100DB000536C656570204C454420746573740A005B
:100DC0000000000000000000000000010204060A0C
:100DD0000F17202C3A4A5D71879DB3C7DAE9F5FCFD
:100DE000FFFCF5E9DAC7B39D87715D4A3A2C2017FD
:100DF0000F0A0604020100000000000000000000CD
:100E000011241FBECFEFDAE0DEBFCDBF04B603FE74
:100E100024C08091F9019091FA01A091FB01B09159
:100E2000FC018730904BA740B04BB9F41092F90108
:100E30001092FA011092FB011092FC0114BE84B7CB
:100E4000877F84BF88E10FB6F8948093600010928A
:100E500060000FBEE0E0FFE3099511E0A0E0B1E023
:100E6000E0EAFBE502C005900D92AA33B107D9F77D
:100E700011E0AAE3B1E001C01D92A93FB107E1F77B
:100E80000E94900F0C94CE2D0C940000FF93EF93D2
:100E9000E0913A01F0913B01309709F00995EF910B
:100EA000FF910895FC018591803011F0EFDFFBCFB9
:100EB0000895FF27E0E230E247FF0CC0419597FF1D
:100EC00009C0EDE26095709580959095611D711D4A
:100ED000811D911D27FF02C0219530E350E2AA2712
:100EE000660F771F881F991FAA1FA41710F0A41B55
:100EF00063955A95A9F7AA3008F0A95FA05DAF9352
:100F0000F395611571058105910541F7ED3211F4F5
:100F1000EF93F395F21718F43F93F395FBCF8F916E
:100F2000B5DFFA95E1F70895E991F991859180305F
:100F300021F0853219F0AADFF9CF089520E0E89476
:100F400055915532C1F3503311F4689455915A3389
:100F500048F4505390F3220F022E220F220F200D3F
:100F6000250FF4CF0EF4219589919991533619F3F9
:100F7000533729F1533559F1BC0188279927E89453
:100F80005C3621F48991999168945591543639F4DD
:100F900046EF7EF077FF0DC08FEF9FEF0AC0553709
:100FA0004AE039F0583540E121F0523642E009F08C
:100FB0000895FF93EF937DDFEF91FF91B7CFFF93FC
:100FC000EF93FC0181918030B9F360DFFBCFFF9399
:100FD000EF9368DFF1CFDF93CF93CDB7DEB72596E0
:100FE000A3DFCF91DF91089561110BC0FC018281D5
:100FF000882321F085EE0E946D1603C085EE0E94C5
:10100000351780E090E0089508956091BC017091DB
:10101000BD018091BE019091BF010E94FD205698B4
:101020005E9825982D9826982E9827982F9881308D
:1010300019F0823021F00895259A2D9A0895269A64
:101040002E9A089585E098E0892B11F00E940508FA
:1010500080E090E0089556985E9825982D982698FF
:101060002E9827982F988FEF90E090938900809387
:10107000880090938B0080938A0090938D008093DA
:101080008C00259A2D9A2FEF80E792E02150804026
:101090009040E1F700C00000269A2E9A2FEF80E7DB
:1010A00092E0215080409040E1F700C00000279A74
:1010B0002F9A2FEF80E792E0215080409040E1F797
:1010C00000C0000025982D982FEF80E792E0215076
:1010D00080409040E1F700C0000026982E982FEF46
:1010E00080E792E0215080409040E1F700C000008E
:1010F00027982F9856985E9825982D9826982E9880
:1011000027982F98089589EA8093800089E080933A
:10111000810024982C983F988AB18F748AB96E9870
:10112000479A8BB1806B8BB9769A0E942B0884E02A
:1011300098E0892B11F00E94040880E090E0089567
:1011400080E28093000180913C0181110EC00E94D9
:10115000EF0881E080933C012FEF83ED90E3215075
:1011600080409040E1F700C0000080E40E94F50854
:101170008093000181112EC00E941F0980930001FD
:10118000811128C00E941F0980930001811122C093
:101190008FE30E941F098093000181111BC00E94F0
:1011A000170980E40E94F50880930001811112C0A4
:1011B0008CE00E941F098093000181110BC00E94E6
:1011C0001F0980930001811105C08FE30E941F0950
:1011D000809300010E9417098091000108951092E8
:1011E000B9008AE08093B800089594EA9093BC0017
:1011F0009091BC0097FFFCCF9091B900987F9830F8
:1012000021F0903111F081E008958093BB0084E8D3
:101210008093BC008091BC0087FFFCCF8091B90017
:10122000887F883111F0803471F780E0089584E977
:101230008093BC008091BC0084FDFCCF0895809316
:10124000BB0084E88093BC008091BC0087FFFCCF8A
:101250009091B900987F81E0983209F480E0089578
:1012600084E88093BC008091BC0087FFFCCF809114
:10127000BB00089580910001811115C080E40E9497
:10128000F5088093000181110CC082E10E941F09C2
:1012900080930001811105C08FEF0E941F09809388
:1012A00000010E94170984B1807F84B985B1807FD5
:1012B00085B98AB1837F8AB98BB1837F8BB93E9818
:1012C000469808950E94A008809300010E943A0960
:1012D00080B38C7080BB81B3836F81BBAEE3B1E020
:1012E000ECE4F1E08EE08E0F11921D928E13FCCF94
:1012F00083E898E0892B11F00C94830808959F925D
:10130000AF92BF92CF92DF92EF92FF920F931F9313
:10131000CF93DF93809100018823E1F080913D011C
:101320008F5F80933D01811115C082E493E00E949C
:1013300052070E94A00880930001882329F088E2C8
:1013400093E00E94520706C084E193E00E94520796
:101350000E942B080EE311E0C0E0D0E0BB24B39460
:1013600082E0A82ECC24C394D12C25E0E22E23E0E9
:10137000F22EC730D10500F580910001811164C0C3
:1013800080E40E94F50880930001811112C082E17F
:101390000E941F098093000181110BC0C6010C2E11
:1013A00001C0880F0A94EAF780950E941F09809374
:1013B00000010E94170948C0CA30A1F028F4C830C3
:1013C00059F0C93061F005C0CC3089F070F0CD30F3
:1013D00089F0209A289810C0219A29980DC0229A45
:1013E0002A980AC0239A2B9807C0529A01C0539A90
:1013F0005B9802C03E9A469890EA9A95F1F79FB1A1
:10140000799902C082E001C080E091709B25982B01
:101410007C9902C084E001C080E0892B7D9902C0E4
:1014200038E001C030E0832B7E9902C020E101C08A
:1014300020E0822B9FB19095991F9927991F929533
:10144000990F907E892B10C080910001811174C08A
:1014500080E40E94F50880930001882309F459C0B4
:10146000912C0E941709892DF8019081981739F164
:10147000808380910101882301F18091D70180FF51
:1014800004C08AE093E00E9452078091D70180FF58
:101490000CC0809101011F928F93FF92EF920E94E6
:1014A000EB070F900F900F900F908091D70180FF66
:1014B00004C083E093E00E945207A09201010E94C1
:1014C0003A0921960F5F1F4FCE30D10509F051CF59
:1014D000809101018823B1F081508093010188231C
:1014E00039F08FE99FE00197F1F700C000000AC0D2
:1014F000ACE4B1E0EEE3F1E0CF01825F91919D9326
:101500008E13FCCF82E298E0892BC1F00E94220862
:1015100015C083E10E941F09809300018111A0CFB3
:1015200081E40E94F50880930001811199CF0E9407
:101530003009982E909495CF80E096CF81E0DF918E
:10154000CF911F910F91FF90EF90DF90CF90BF90C0
:10155000AF909F900895E82FF0E0E45BFE4F80810C
:101560000895CF92DF92EF92FF920F931F93CF9344
:10157000DF938CEE92E00E9452078CE4E82E81E02B
:10158000F82EC0E0D0E097EEC92E92E0D92E0EEDF5
:1015900012E0DF93CF93DF92CF920E94EB0784EEAD
:1015A00092E00E945207F70181917F0190E00E9432
:1015B00063219F938F931F930F930E94EB078CEDF2
:1015C00092E00E94520721968DB79EB708960FB6FB
:1015D000F8949EBF0FBE8DBFCE30D105D1F6DF91FE
:1015E000CF911F910F91FF90EF90DF90CF900895D2
:1015F0008B3B910578F4883A910540F5853A910541
:10160000D0F48430910508F0B1C08130910509F41F
:10161000ADC06BC0803E910508F467C0883E91055F
:1016200008F4A4C09C01205F31092031310508F085
:101630005CC090650895853A910509F459C0863AD1
:10164000910509F058C082E890E40895883A910520
:1016500009F454C0893A910509F453C08A3A9105B6
:1016600009F452C08B3A910509F451C08C3A9105A6
:1016700009F450C08D3A910509F44FC0803B9105A3
:1016800009F44EC08E3A910509F44DC08F3A910588
:1016900009F44CC0813B910509F44BC0823B910594
:1016A00009F44AC0833B910509F449C0843B910584
:1016B00009F448C0853B910509F447C0863B910574
:1016C00009F446C0873B910509F445C0883B910564
:1016D00009F444C0893B910509F443C08A3B910554
:1016E00009F442C080E094E4089580E090E0089519
:1016F00081E890E4089583E890E4089582EE94E40C
:10170000089589EE94E408958AEE94E4089585EBB3
:1017100094E4089586EB94E4089587EB94E40895A7
:101720008CEC94E408958DEC94E4089583E895E4BA
:1017300008958AE895E4089582E995E4089584E996
:1017400095E4089581E296E4089583E296E408958D
:1017500084E296E4089585E296E4089586E296E4AC
:10176000089587E296E408958AE296E4089508953C
:1017700096E0799FF001112494E5899FE00DF11D19
:101780001124E60FF11DEE0FFF1FEC51FF4F859165
:1017900094910895880F991FFC01E05AF0408591BB
:1017A00094910895880F991FFC01E052FF4F859195
:1017B0009491089526E0729FF001112444E5849FDE
:1017C000E00DF11D1124E60FF11DEE0FFF1FEC518E
:1017D000FF4F859194919C013A9521154FE1340773
:1017E00008F41EC13F512115304120F49F700E9422
:1017F000D20B08959C0130532115304118F49927DC
:10180000906C0895811520E5920769F40E94BD1A35
:101810004FEF84E39CE0415080409040E1F700C0EE
:1018200000000C941F22813020E5920751F48CE5D2
:1018300093E00E9452078091D70181608093D70185
:1018400008959C0130552115304108F051C0292FD1
:1018500033272F70332721303105D9F4AC01437081
:10186000552702C0220F331F4A95E2F73C68AC01AE
:1018700064E0440F551F6A95E1F744275370242B09
:10188000352B73E0880F991F7A95E1F780769927B9
:101890001DC02230310529F4982F8827816F906A66
:1018A000089523303105A9F4AC014370552721E098
:1018B00030E002C0220F331F4A95E2F73C6843E054
:1018C000880F991F4A95E1F7807E9770822B932BA2
:1018D000089524303105E1F4AC014370552721E02F
:1018E00030E002C0220F331F4A95E2F73A68E7CF93
:1018F0009C0130572115304118F49F709062089573
:101900009C0130582115304118F49F70906A089559
:10191000803E9105E0F4803C910558F581339105B6
:1019200009F46FC048F48932910509F463C08A3222
:10193000910509F46DC072C089339105E9F08238D0
:101940009105D1F08533910509F44DC067C0833E00
:10195000910581F138F4803E9105B9F0823E910500
:10196000D9F05CC0863E910561F1873E9105A1F1F9
:1019700055C00E94CA0B08952091EA0120FD02C0C3
:1019800021FF4CC080EE90E049C08091EA0180FFC9
:10199000F9CF89E390E042C08091EA0182FF0EC056
:1019A0008091EA0184FF03C080E090E037C083EEBD
:1019B00090E034C08091EA0182FFF2CF82EE90E0A5
:1019C0002DC08091EA0183FF0BC08091EA0184FD64
:1019D000EBCF87EE90E022C08091EA0183FFF5CF44
:1019E00086EE90E01BC08091EA0185FF07C089E286
:1019F00090E014C08091EA0185FFF9CF85E390E083
:101A00000DC08091EA0186FF07C08AE290E006C01F
:101A10008091EA0186FFF9CF81E390E00E94F80A05
:101A20000895089580916D0108959FB7F8941092DC
:101A30005C019FBF9091F001943009F057C09091E4
:101A4000E9009F703091EC00232F217030FD20E8D9
:101A5000922B24E02093E9002091EB0020FF43C06B
:101A60002091EE0027FF3FC020915A01222321F050
:101A70002091E80025FF37C010925A0126E03091EE
:101A8000E80035FD15C03091F001343061F530913A
:101A9000EB0035FD28C0215021F481E080935A01EC
:101AA00022C0EFE9FFE03197F1F700C00000E7CF77
:101AB0008093F1008091E80085FD0AC08091E800E4
:101AC00080FFFCCF8091E8008E778093E80006C00D
:101AD0008FB7F89421E020935C018FBF9F709093A3
:101AE000E90080E008959F709093E9008FEF0895DA
:101AF000CF93DF9300D01F92CDB7DEB79C018091CA
:101B0000F001843019F593E099833B832A83909305
:101B1000E9008FEF9091E800815095FD06C095EDAA
:101B20009A95F1F700008111F5CF8091E80085FFCB
:101B30000DC040E050E063E070E0CE0101960E94ED
:101B400048108091E8008E778093E8000F900F9006
:101B50000F90DF91CF910895CF93DF9300D01F9224
:101B6000CDB7DEB72091F001243021F522E02983A2
:101B70009B838A8383E08093E9008FEF9091E80054
:101B8000815095FD06C095ED9A95F1F70000811101
:101B9000F5CF8091E80085FF0DC040E050E063E0A4
:101BA00070E0CE0101960E9448108091E8008E7787
:101BB0008093E8000F900F900F90DF91CF910895E0
:101BC0002091F0012430F1F422E02093E9002FEF7E
:101BD0003091E800215035FD06C035ED3A95F1F71A
:101BE00000002111F5CF2091E80025FF0BC040E057
:101BF00050E065E070E00E9448108091E8008E7728
:101C00008093E8000895CF93DF932091F001243072
:101C100009F048C0EC0180910C018823E1F080912B
:101C20000D018823C1F085E08093E9008FEF90914A
:101C3000E800815095FD06C095E19A95F1F7000006
:101C40008111F5CF8091E80085FF2CC040E050E085
:101C500060E170E017C081E08093E9008FEF909120
:101C6000E800815095FD06C095ED9A95F1F70000CA
:101C70008111F5CF8091E80085FF14C040E050E06D
:101C800068E070E0CE010E9448108091E8008E77F5
:101C90008093E80080E1FE01ADE5B1E001900D9296
:101CA0008A95E1F7DF91CF91089583E993E00E944F
:101CB00052078091EF01811109C00E94DD110E943D
:101CC0003A128091E20084608093E20008958FE8E8
:101CD00093E00E9452071092EF0108958BE893E081
:101CE0000C94520787E893E00E9452070C94EF2B64
:101CF00083E893E00E9452070E94B9210E94F52BCD
:101D00000E94DF140C94110D20915B012F5F822F34
:101D100062E30E94632D992319F020935B010895DB
:101D200010925B0180915C01882371F18091F00138
:101D3000843041F58091E9008F702091EC00922F62
:101D4000917020FD90E8892B94E09093E9009091A8
:101D5000EB0090FF14C09091EE0097FF10C090919F
:101D6000E80095FF03C01092F100F9CF9091E800D0
:101D700090FF05C09091E8009E779093E8008F70E7
:101D80008093E90010925C01089542E061EC81E0EB
:101D90000E94571142E061EC82E00E94571142E03C
:101DA00061EC83E00E94571142E261EC84E00E9402
:101DB000571142E161EC85E00C9457118091F201DA
:101DC000833009F455C030F4813071F0823009F469
:101DD0008EC008958A3009F47AC08B3009F460C04F
:101DE000893009F09CC020C08091F101813A09F04E
:101DF00096C08091E800877F8093E8008091F5018C
:101E00009091F601892B21F460E18DE591E003C00A
:101E100060E080E090E070E00E9493108091E80024
:101E20008B778093E80008958091F101813209F069
:101E300076C08091F5019091F601009719F0049712
:101E400009F06DC08091E800877F8093E800809161
:101E5000E80082FD05C08091F0018111F8CF5FC0DC
:101E60008091F10080936D018091E8008B7753C0E1
:101E70008091F101813A09F052C08091F501909171
:101E8000F601892B09F04BC08091E800877F809391
:101E9000E8008091E80080FFFCCF80910C0136C003
:101EA0008091F1018132D9F58091F5019091F6018F
:101EB000892BA9F58091E800877F8093E8000E9434
:101EC0008C118091F30180930C010C94BD1A8091C8
:101ED000F101813221F58091E800877F8093E8004D
:101EE0000E948C118091F40180936E01089580917D
:101EF000F101813AA1F48091E800877F8093E800A6
:101F00008091E80080FFFCCF80916E018093F1000A
:101F10008091E8008E778093E8000C948C110895EE
:101F200084B7877F84BF88E10FB6F8948093600000
:101F3000109260000FBE90E080E80FB6F894809396
:101F40006100909361000FBE0E946C150E94DD112C
:101F50000E943A128091E20084608093E20085E161
:101F60009DE00E94F82078940E94BF140E946E1594
:101F700082E091E00E94DA140E94DD2B82E793E078
:101F80000E9452078091F001853089F48EE693E03B
:101F90000E9452070E947D218091EE01882391F3D7
:101FA0000E94A521882371F30E943210EBCF0E947A
:101FB0009C15E8CF292F332723303105C9F064F46D
:101FC0002130310581F02230310509F043C08DE820
:101FD00090E02BEC33E042C021323105F1F02232A7
:101FE000310541F137C082E190E028E534E036C0A8
:101FF00099278130910541F08230910541F0892B7C
:1020000049F5E7ECF3E005C0EFEAF3E002C0E7E9E9
:10201000F3E0849190E09F0121C06530D8F4E62F71
:10202000F0E0EE0FFF1FEB5DFE4F2081318189E074
:1020300090E014C0653070F470E0FB01EE0FFF1FFC
:10204000E55EFE4F20813181FB01EA5EFE4F80811B
:1020500090E004C080E090E020E030E0FA013183BD
:102060002083089580E189BD82E189BD09B400FE25
:10207000FDCF8091D8008F7D8093D8008091E000C3
:1020800082608093E0008091E00081FDFCCF0895A4
:10209000CF92DF92EF92FF920F931F93CF93DF9334
:1020A000EC018B016A010E94AB11811133C0C11494
:1020B000D10439F0F60180819181081B190BC80FFA
:1020C000D91FE12CF12C0115110519F18091E800BF
:1020D00085FD16C08091E8008E778093E800C114DA
:1020E000D10449F0F60180819181E80EF91EF18258
:1020F000E08285E00FC00E94AB11882321F30AC063
:1021000089918093F10001501109FFEFEF1AFF0A46
:10211000DACF80E0DF91CF911F910F91FF90EF9088
:10212000DF90CF9008952091F7013091F8012617A4
:10213000370748F06115710539F42091E8002E77D2
:102140002093E80001C0B90140E061157105A9F1D3
:102150002091F001222309F443C0253009F442C044
:102160002091E80023FD40C02091E80022FD32C00C
:102170002091E80020FFE9CF4091F3002091F20088
:1021800030E0342BFC01CF016115710559F0283086
:10219000310540F481918093F100615071092F5F06
:1021A0003F4FF1CF41E02830310509F040E0209168
:1021B000E8002E772093E800C8CF4111C9CF0AC0AC
:1021C0008091F001882361F0853061F08091E80012
:1021D00083FD0AC08091E80082FFF2CF80E008957D
:1021E00082E0089583E0089581E008952091F70149
:1021F0003091F8012617370748F06115710539F459
:102200002091E8002E772093E80001C0B901FC017D
:1022100020E06115710591F18091F001882309F4A6
:1022200040C0853009F43FC08091E80083FD3DC087
:102230008091E80082FD2FC08091E80080FFE9CF07
:102240002091F3008091F20090E0922B61157105CE
:1022500059F08830910540F424912093F100319693
:10226000615071090196F2CF21E0089709F020E052
:102270008091E8008E778093E800CBCF2111CCCFFE
:102280000AC08091F001882361F0853061F080916F
:10229000E80083FD0AC08091E80082FFF2CF80E071
:1022A000089582E0089583E0089581E00895982FCD
:1022B000973058F59093E900981739F07091EC0039
:1022C0002091ED005091F00003C0242F762F50E0B4
:1022D00021FF19C03091EB003E7F3093EB0030912D
:1022E000ED003D7F3093ED003091EB003160309395
:1022F000EB007093EC002093ED005093F0002091E0
:10230000EE0027FF07C09F5FD3CF8F708093E90057
:1023100081E0089580E008958091F10187FF11C068
:102320008091E80082FD05C08091F0018111F8CF15
:1023300011C08091E8008B770BC08091F001882359
:1023400049F08091E80080FFF8CF8091E8008E7717
:102350008093E80008952091E4003091E50095E62F
:102360004091EC00842F817040FF22C08091E800F2
:1023700080FD1CC08091F001882391F0853091F0A0
:102380008091EB0085FD10C04091E4005091E50084
:102390004217530729F39A01915011F784E00895E9
:1023A00082E0089583E0089581E0089580E0089533
:1023B0004091E80042FFDECF08950E944B120E9438
:1023C0005312E0EEF0E0808181608083E8EDF0E080
:1023D00080818F77808319BCA7EDB0E08C918E7FD0
:1023E0008C9380818F7E80831092EF0108950F93EC
:1023F0001F93CF93DF930E944B120E945312C8ED9C
:10240000D0E088818F7788838881806888838881FD
:102410008F7D888319BC1092F0011092EC0110920C
:10242000EE011092ED0100EE10E0F80180818B7F4B
:10243000808388818160888342E060E080E00E9440
:102440005711E1EEF0E080818E7F8083E2EEF0E0D4
:10245000808181608083808188608083F8018081B1
:102460008E7F8083888180618883DF91CF911F91E7
:102470000F910895E8EDF0E080818F7E8083E7ED95
:10248000F0E080818160808384E082BF81E080937E
:10249000EF010C94F711E8EDF0E080818E7F8083EE
:1024A0001092E20008951092DA001092E10008956F
:1024B0001F920F920FB60F9211242F933F934F93B9
:1024C0005F936F937F938F939F93AF93BF93EF939C
:1024D000FF938091E10082FF0BC08091E20082FFB8
:1024E00007C08091E1008B7F8093E1000E94840E01
:1024F0008091DA0080FF1FC08091D80080FF1BC050
:102500008091DA008E7F8093DA008091D90080FF7D
:102510000DC080E189BD82E189BD09B400FEFDCF17
:1025200081E08093F0010E94550E05C019BC109205
:10253000F0010E94670E8091E10080FF19C0809138
:10254000E20080FF15C08091E2008E7F8093E20060
:102550008091E20080618093E2008091D8008062E7
:102560008093D80019BC85E08093F0010E94720E20
:102570008091E10084FF30C08091E20084FF2CC094
:1025800080E189BD82E189BD09B400FEFDCF809163
:10259000D8008F7D8093D8008091E1008F7E80935A
:1025A000E1008091E2008F7E8093E2008091E20062
:1025B00081608093E2008091EC01882311F084E037
:1025C00007C08091E30087FD02C081E001C083E085
:1025D0008093F0010E94780E8091E10083FF29C072
:1025E0008091E20083FF25C08091E100877F809386
:1025F000E10082E08093F0011092EC018091E10013
:102600008E7F8093E1008091E2008E7F8093E200D4
:102610008091E20080618093E20042E060E080E02F
:102620000E9457118091F00088608093F0000E9412
:102630006E0EFF91EF91BF91AF919F918F917F911E
:102640006F915F914F913F912F910F900FBE0F901F
:102650001F9018951F920F920FB60F9211242F936F
:102660003F934F935F936F937F938F939F93AF931A
:10267000BF93CF93DF93EF93FF93C091E900CF70A7
:102680008091EC00D82FD17080FDD0E81092E90045
:102690008091F000877F8093F00078940E946E1301
:1026A0001092E9008091F00088608093F000CD2BBB
:1026B000CF70C093E900FF91EF91DF91CF91BF916F
:1026C000AF919F918F917F916F915F914F913F91CA
:1026D0002F910F900FBE0F901F9018951F93CF93BF
:1026E000DF93CDB7DEB7AA970FB6F894DEBF0FBE63
:1026F000CDBFE1EFF1E088E08E0F9091F100919372
:102700008E13FBCF0E94DE0E8091E80083FF1FC175
:102710008091F1019091F201492F50E04A3051052A
:1027200008F015C1FA01EA5AFF4F0C94832D803846
:1027300081F0823809F00BC18091F5018F70809390
:10274000E9008091EB0085FB882780F91092E90071
:1027500006C08091ED019091EE01911182609091FF
:10276000E800977F9093E8008093F1001092F100C9
:10277000C8C0282F2D7F09F0EAC0882319F08230C5
:1027800061F0E5C08091F301813009F0E0C0933041
:1027900009F080E08093EE012BC08091F30181115C
:1027A00027C08091F5018F7009F4D1C08093E900B2
:1027B0002091EB0020FF1CC0933021F48091EB00AE
:1027C000806214C09091EB0090619093EB0021E047
:1027D00030E0A90102C0440F551F8A95E2F74093EB
:1027E000EA001092EA008091EB0088608093EB0091
:1027F0001092E9008091E800877F86C08111A7C010
:102800001091F3011F778091E3008078812B8093F2
:10281000E3008091E800877F8093E8000E948C119C
:102820008091E80080FFFCCF8091E3008068809376
:10283000E300111102C082E001C083E08093F00147
:1028400086C08058823008F082C08091F301909158
:10285000F4018C3D53E0950779F583E08A838AE2A1
:1028600089834FB7F894DE01139620E03EE051E2F1
:10287000E32FF0E050935700E49120FF03C0E2956E
:10288000EF703F5FEF708E2F90E0EA3010F0C79648
:1028900001C0C0968D939D932F5F243149F74FBFA0
:1028A0008091E800877F8093E8006AE270E0CE01C3
:1028B00001960E94931014C0AE014F5F5F4F60916C
:1028C000F5010E94DA0FBC01892B09F440C09091F8
:1028D000E800977F9093E80089819A810E94F61022
:1028E0008091E8008B778093E80031C0803879F5DB
:1028F0008091E800877F8093E8008091EC018093CD
:10290000F1008091E8008E778093E8000E948C119E
:102910001EC081111CC09091F3019230C0F48091CF
:10292000E800877F8093E8009093EC010E948C116F
:102930008091EC01811106C08091E30087FD02C007
:1029400081E001C084E08093F0010E94C50E809177
:10295000E80083FF0AC08091E800877F8093E80049
:102960008091EB0080628093EB00AA960FB6F894FA
:10297000DEBF0FBECDBFDF91CF911F910895CF93E2
:102980008091F0018823A1F0C091E900CF7090916F
:10299000EC00892F817090FD80E8C82B1092E9002F
:1029A0008091E80083FD0E946E13CF70C093E90010
:1029B000CF91089590937401809373010895E091ED
:1029C0007301F0917401309721F00190F081E02DB6
:1029D000099480E00895EF92FF920F931F93CF9395
:1029E000DF93E0917301F09174013097B1F18C01A4
:1029F0000280F381E02D09958091D70182FF2DC0DF
:102A000080FF04C08DE895E00E945207E80110E1C4
:102A100087E8E82E85E0F82E8091D70180FF0BC073
:102A200088811F928F93FF92EF920E94EB070F9085
:102A30000F900F900F90115021961111EDCF8091B2
:102A4000D70180FF0AC085E895E0DF91CF911F9103
:102A50000F91FF90EF900C945207DF91CF911F914F
:102A60000F91FF90EF900895E0917301F091740140
:102A7000309721F00480F581E02D0994089520918C
:102A80007101309172018217930771F09093720176
:102A900080937101E0917301F0917401309721F0FE
:102AA0000680F781E02D0994089520916F013091FF
:102AB00070018217930771F09093700180936F01FA
:102AC000E0917301F0917401309721F00084F18559
:102AD000E02D0994089508950C946B150E94BB2174
:102AE0000E9462090C948122CF93C82F8091D70154
:102AF00082FF1EC080FF04C086EA95E00E94520754
:102B00008091D70180FF0CC01F92CF9381EA95E09E
:102B10009F938F930E94EB070F900F900F900F9051
:102B20008091D70180FF04C08FE995E00E94520791
:102B30008C2FCF910C94110DCF92DF92EF92FF92D8
:102B40000F931F93CF93DF93CDB7DEB72B970FB6BD
:102B5000F894DEBF0FBECDBF0E947F0986E7C82E66
:102B600081E0D82E00E010E0E02E802F0E94AB0A1A
:102B7000F60141916F01F42EF826B1F40F5F1F4F5B
:102B80000E30110589F78FEF89838A831B820E949B
:102B9000C4218160782F9D838C8349815A816B8108
:102BA0008D810E943F1640C09091D70191FF04C0D3
:102BB0008B870E94B10A8B8520E030E04F2D50E0DA
:102BC000922FBA01022E02C0759567950A94E2F71A
:102BD00060FF24C02E83EF8221E030E0690102C053
:102BE000CC0CDD1C9A95E2F790E08C219D21892B7D
:102BF00009F420E028870E94C4218160782F9A87F9
:102C000089874E815F8168858A850E943F16F80119
:102C1000EA58FE4F8081C826C08206C02F5F3F4F12
:102C20002630310569F6AACF0E94F2251091750170
:102C30000E94DF141817A1F00E94DF148093750121
:102C40002B960FB6F894DEBF0FBECDBFDF91CF91AC
:102C50001F910F91FF90EF90DF90CF900C9474151F
:102C60002B960FB6F894DEBF0FBECDBFDF91CF918C
:102C70001F910F91FF90EF90DF90CF900895CF9329
:102C8000DF93CDB7DEB72B970FB6F894DEBF0FBE3C
:102C9000CDBF4F83588769877A878B87DE0111966E
:102CA00086E0FD0111928A95E9F785E0FE013796ED
:102CB00001900D928A95E1F749815A816B817C815F
:102CC0008D819E810E94571D2B960FB6F894DEBF12
:102CD0000FBECDBFDF91CF910895CF93882309F424
:102CE000C2C0C82F823859F40E94DF1481FDBBC0D6
:102CF00089E30E94F31F0E94D22089E30CC083382D
:102D000079F40E94DF1480FDAEC083E50E94F31FBA
:102D10000E94D22083E50E944620CF910C94D220BD
:102D2000843859F40E94DF1482FD9DC087E40E941C
:102D3000F31F0E94D22087E4EECF8CEF8C0F813AF4
:102D400048F48C2F0E94852A81118DC08C2F0E94FF
:102D5000F31FE3CF80E28C0F883048F4C77081E026
:102D600001C0880FCA95EAF70E949B20D6CF8BE559
:102D70008C0F833078F4C53A29F0C63A31F083E8F5
:102D800090E005C081E890E002C082E890E0CF9139
:102D90000C943F1588E58C0F833108F064C0C83A65
:102DA00039F1C93A41F1CA3A49F1CB3A51F1CC3A39
:102DB00059F1CD3A61F1C03B69F1CE3A71F1CF3AA8
:102DC00079F1C13B81F1C23B89F1C33B91F1C43B35
:102DD00099F1C53BA1F1C63BA9F1C73BB1F1C83B95
:102DE000B9F1C93BC1F1CA3BC9F180E090E038C0FC
:102DF00082EE90E035C089EE90E032C08AEE90E03D
:102E00002FC085EB90E02CC086EB90E029C087EBCB
:102E100090E026C08CEC90E023C08DEC90E020C0C8
:102E200083E891E01DC08AE891E01AC082E991E050
:102E300017C084E991E014C081E292E011C083E2FE
:102E400092E00EC084E292E00BC085E292E008C0FE
:102E500086E292E005C087E292E002C08AE292E058
:102E6000CF910C945515CF910895882309F44BC048
:102E7000823859F40E94DF1481FF45C089E30E9423
:102E8000F31F0E94D22089E30CC0833871F40E94A2
:102E9000DF1480FF38C083E50E94F31F0E94D22018
:102EA00083E50E9446200C94D220843859F40E9475
:102EB000DF1482FF28C087E40E94F31F0E94D22003
:102EC00087E4EFCF9CEF980F913A58F390E2980F78
:102ED000983050F4877091E001C0990F8A95EAF715
:102EE000892F0E94A120DFCF9BE5980F933020F41B
:102EF00080E090E00C943F15885A833120F480E004
:102F000090E00C9455150895882321F00E949B2091
:102F10000C94D2200895882321F00E94A1200C94C3
:102F2000D2200895BF92CF92DF92EF92FF920F933B
:102F30001F93CF93DF9300D000D000D0CDB7DEB782
:102F400025E0FC01DE01119601900D922A95E1F732
:102F5000FC01408131810281258122952F7063819E
:102F60007481672B09F4E7C23F3F19F44F3F09F41E
:102F7000E2C27C0149833A8389819A812E830E942F
:102F8000B21F182FB92E0E94B11F0E94781EEB2D80
:102F9000E295EF70F0E0E05AFF4F2E810C94832D04
:102FA0008B2D807F9B2D9F70F92E882319F0F29432
:102FB00080EFF822002349F0FF2009F469C28F2D29
:102FC0000E94AB200E94D22063C2812F0E9435173D
:102FD000FF2009F4B0C28F2D0E94B12026960FB6B3
:102FE000F894DEBF0FBECDBFDF91CF911F910F913F
:102FF000FF90EF90DF90CF90BF900C94D2203B2DAC
:10300000307F8B2D8F70303211F08295807F1123AD
:1030100019F0113021F12DC00023B9F0222309F459
:10302000A1C1213009F09EC126960FB6F894DEBFEB
:103030000FBECDBFDF91CF911F910F91FF90EF9009
:10304000DF90CF90BF900C94BB20222319F0213049
:1030500009F471C28E830E94BE208E8197C1002325
:1030600021F0263008F067C27DC1253008F063C228
:103070008DC1002321F0222309F474C109C2222347
:1030800009F484C11AC22B2D26952695237030E0B1
:103090002115310521F021303105D1F04CC200233A
:1030A00021F0812F9B2D937002C080E090E0269646
:1030B0000FB6F894DEBF0FBECDBFDF91CF911F9149
:1030C0000F91FF90EF90DF90CF90BF900C943F1541
:1030D000002321F0812F9B2D937002C080E090E0AF
:1030E00026960FB6F894DEBF0FBECDBFDF91CF910D
:1030F0001F910F91FF90EF90DF90CF90BF900C94B5
:103100005515812F002319F00E94782402C00E94D7
:10311000E02426960FB6F894DEBF0FBECDBFDF9138
:10312000CF911F910F91FF90EF90DF90CF90BF90C4
:103130000C9465258B2D837009F07BC00111FBC1B8
:10314000812F829586958770880F880F912F9F70A9
:10315000C92ED12CE12CF12C082E04C0CC0CDD1C86
:10316000EE1CFF1C0A94D2F714FF12C04FE050E08F
:1031700060E070E004C0440F551F661F771F8A95FA
:10318000D2F7CB01BA01609570958095909503C0F8
:1031900060E070E0CB012B2D269526952370422F01
:1031A00050E042305105D9F04330510569F16C29A6
:1031B0007D298E299F294130510551F126960FB660
:1031C000F894DEBF0FBECDBFDF91CF911F910F915D
:1031D000FF90EF90DF90CF90BF900C949F1E6C29D2
:1031E0007D298E299F2926960FB6F894DEBF0FBE43
:1031F000CDBFDF91CF911F910F91FF90EF90DF90A6
:10320000CF90BF900C94BB1E0E949F1EC701B601B9
:1032100026960FB6F894DEBF0FBECDBFDF91CF91DB
:103220001F910F91FF90EF90DF90CF90BF900C9483
:10323000831E002319F08B2D817001C08695882391
:1032400009F479C1812F829586958770880F880F40
:10325000912F9F70C92ED12CE12CF12C082E04C087
:10326000CC0CDD1CEE1CFF1C0A94D2F714FF12C01C
:103270004FE050E060E070E004C0440F551F661F4F
:10328000771F8A95D2F7CB01BA016095709580952A
:10329000909503C060E070E0CB012B2D269526951C
:1032A0002370422F50E042305105D9F04330510590
:1032B00069F16C297D298E299F294130510551F1F1
:1032C00026960FB6F894DEBF0FBECDBFDF91CF912B
:1032D0001F910F91FF90EF90DF90CF90BF900C94D3
:1032E000791F6C297D298E299F2926960FB6F8947F
:1032F000DEBF0FBECDBFDF91CF911F910F91FF9029
:10330000EF90DF90CF90BF900C94951F0E94791F93
:10331000C701B60126960FB6F894DEBF0FBECDBF2B
:10332000DF91CF911F910F91FF90EF90DF90CF90A1
:10333000BF900C945D1F103FD1F118F4103E50F473
:10334000A2C0123F09F464C008F44DC0133F09F451
:1033500074C099C01F708B2D8F710023A1F00E9443
:10336000F61E812F26960FB6F894DEBF0FBECDBF96
:10337000DF91CF911F910F91FF90EF90DF90CF9051
:10338000BF900C9484170E94171F812F26960FB6AA
:10339000F894DEBF0FBECDBFDF91CF911F910F918B
:1033A000FF90EF90DF90CF90BF900C948B1700238D
:1033B000B1F0253008F0BFC08B2D8F7126960FB667
:1033C000F894DEBF0FBECDBFDF91CF911F910F915B
:1033D000FF90EF90DF90CF90BF900C943C1F263071
:1033E00008F0A9C0E9CF0023A9F08B2D8F71269694
:1033F0000FB6F894DEBF0FBECDBFDF91CF911F9106
:103400000F91FF90EF90DF90CF90BF900C94F61E3D
:10341000002359F38B2D8F7126960FB6F894DEBFDB
:103420000FBECDBFDF91CF911F910F91FF90EF9015
:10343000DF90CF90BF900C94171F002399F08B2D35
:103440008F7126960FB6F894DEBF0FBECDBFDF9109
:10345000CF911F910F91FF90EF90DF90CF90BF9091
:103460000C94E11E26960FB6F894DEBF0FBECDBFBA
:10347000DF91CF911F910F91FF90EF90DF90CF9050
:10348000BF900C94D71E0023A9F0222309F4ADCFDE
:10349000812F26960FB6F894DEBF0FBECDBFDF9109
:1034A000CF911F910F91FF90EF90DF90CF90BF9041
:1034B0000C946D16222309F4ADCF812F26960FB6FA
:1034C000F894DEBF0FBECDBFDF91CF911F910F915A
:1034D000FF90EF90DF90CF90BF900C9435174B2D5D
:1034E0004F70612FC7010E94F40726960FB6F8941B
:1034F000DEBF0FBECDBFDF91CF911F910F91FF9027
:10350000EF90DF90CF90BF900C94FB1D4B2D4F7030
:10351000612FC70126960FB6F894DEBF0FBECDBF50
:10352000DF91CF911F910F91FF90EF90DF90CF909F
:10353000BF900C94B70B26960FB6F894DEBF0FBE63
:10354000CDBFDF91CF911F910F91FF90EF90DF9052
:10355000CF90BF9008950E94B8200E948D200E94B5
:10356000D2200E9498260E94652580E090E00E946B
:103570003F1580E090E00C9455150E94A8200C9413
:10358000AB1A0E94B21F292F22952F7030E02C30E9
:1035900031054CF42A3031056CF4225031092230C7
:1035A000310588F407C02C30310549F02F30310542
:1035B00031F009C0803E48F0803F29F406C093FBFB
:1035C000882780F9089580E0089581E00895CF93D9
:1035D000DF9300D000D01F92CDB7DEB70F900F90D1
:1035E0000F900F900F90DF91CF910895CF93DF93BD
:1035F00000D000D000D0CDB7DEB726960FB6F89435
:10360000DEBF0FBECDBFDF91CF9108951F93CF9343
:10361000DF93C091840116E080918501C81799F06D
:10362000D0E01C9FF0011D9FF00D1124EA57FE4FC2
:103630004081518162817381848195810E94F61A53
:103640002196C770E9CFDF91CF911F9108954091E6
:10365000B6015091B7016091B8017091B9018091A4
:10366000BA019091BB010C94F61A8091BB0182952E
:103670008F7009F054C08091B801882309F44FC0BD
:1036800080918401A09185016091B6017091B7018C
:103690004091B9015091BA01B6E08A1709F43FC0D0
:1036A00090E041155105C1F17F3F11F46F3FA1F149
:1036B000B89FF001B99FF00D1124EA57FE4F218108
:1036C00072132AC02081621327C02281211124C0D5
:1036D000238134812417350710F421503109241B2C
:1036E000350B283C3105C0F42091BB012F702061BF
:1036F0002093BB0126E0289FF001299FF00D1124A3
:10370000E557FE4F80818F708061808386EB91E06A
:103710000E9492170C94061B01968770BECF0895E5
:10372000CF92DF92EF92FF920F931F93CF93DF938D
:10373000CDB7DEB762970FB6F894DEBF0FBECDBF30
:103740008C0185E0F801DE011D9601900D928A95AD
:10375000E1F7D8014C9111965C91119712966C91FA
:1037600012971396CD90DC9014973091B60170911A
:10377000B7018091B9019091BA01009709F46BC12A
:103780007F3F19F43F3F09F466C1E090B801EE2095
:1037900009F4C0C02091BB01C816D90628F0F60173
:1037A000E81BF90BCF0104C0809590958C0D9D1DF1
:1037B000FF24F394883C910578F0F12C207F09F0E8
:1037C000C6C07C2DD98AC88A89890E94E71A86EBEF
:1037D00091E00E949217B1C0822F807F09F046C00D
:1037E000751314C0341312C0611110C02F70206102
:1037F0002093BB010E94271B86EB91E00E94921749
:103800008091BB01D80115968C932EC0CD2819F15B
:103810005F3F11F44F3FF9F0F62E61111CC080910B
:1038200084012091850136E0821709F45AC090E0A6
:10383000389FF001399FF00D1124EA57FE4F718136
:10384000571306C07081471303C07281711103C002
:1038500001968770E9CFF62E662309F418C180918E
:10386000BB0181608093BB01F12C11C1751308C0AD
:10387000341306C0611104C08091BB01D801C3C0DC
:103880004D875E878D859E856A8B0E94C11A6A89E5
:103890008823E1F16623D1F12091BB01822F82952B
:1038A0008F7090E0029774F08091B6019091B7010B
:1038B00098878F831986DB86CA862C87CE01079668
:1038C0000E94921786E0F801A6EBB1E001900D92FC
:1038D0008A95E1F70E94351B0E94271BFF24F39471
:1038E000D6C04D875E878D859E850E94B21F292F89
:1038F00022952F7030E0223031050CF0BCC09F7053
:1039000009F0B6C0805E883008F4C1C0C8010E94CA
:103910009217E4CFC816D90608F453C0F601E81B85
:10392000F90BCF01883C910508F450C0F12C7C2D97
:10393000D98AC88A89890E94E71AE6EBF1E086E015
:10394000DF011D928A95E9F70E94271BA0C075131D
:1039500014C0341312C0611110C08091BB01F80172
:103960008583C8010E94921786E0E6EBF1E0DF0153
:103970001D928A95E9F7FE2C8AC04D875E878D855A
:103980009E856A8B0E94C11A6A89882309F4BECF7A
:10399000662309F4BBCF2091BB01822F82958F70E3
:1039A00090E002970CF48ECF8091B6019091B70110
:1039B0009A8389831B82DD82CC822E83CE0101967D
:1039C0007FCF809590958C0D9D1DACCFF62E6623F4
:1039D00009F49CCF75132EC034132CC02091BB0169
:1039E00020FD1FC0822F82958F70D9F0D8011596C7
:1039F0002C9315978F3049F08F5F982F9295907F79
:103A0000822F8F70892B15968C93C8010E94921774
:103A100086E0F801A6EBB1E001900D928A95E1F7FE
:103A200093CF86E0F801A6EBB1E001900D928A9564
:103A3000E1F72DC04D875E878D859E850E94C11A56
:103A4000811140CF8091BB0181608093BB01C8018F
:103A50000E9492171CC0662309F458CF4D875E87D9
:103A60008D859E850E94C11A882309F44FCF2ACFE5
:103A7000811148CF0CC0243031050CF047CF9F7026
:103A800009F440CFF8019581907F09F03BCF8F2D4D
:103A900062960FB6F894DEBF0FBECDBFDF91CF9117
:103AA0001F910F91FF90EF90DF90CF9008951F939B
:103AB000CF93DF93CDB7DEB72C970FB6F894DEBF68
:103AC0000FBECDBF4F83588769877A878B879C87C6
:103AD000CE0107960E94901B882369F08F819885FC
:103AE0002A853B85232BF1F19F3F09F063C08F3F6F
:103AF00009F060C037C086E0FE013796DE011196FE
:103B000001900D928A95E1F76F817885EA85FB85B2
:103B1000309741F17F3F11F46F3F21F120918501F2
:103B200030E0C9010196877099274091840150E0E7
:103B30008417950709F447C069837A83FD83EC8372
:103B400096E0929FD001939FB00D1124AA57BE4FCB
:103B5000FE01319601900D929A95E1F780938501CF
:103B60000E94061B16E080918401909185018917BF
:103B7000C1F1189FC00111248A579E4F0E94901BCB
:103B8000882379F1E09184011E9FF0011124EA5706
:103B9000FE4F4081518162817381848195810E94B1
:103BA000F61A8091840190E001968770992780939E
:103BB0008401D9CF4F81588569857A858B859C850D
:103BC0000E94F61ACFCF0E94BD1A10928501109262
:103BD0008401E6EBF1E086E0DF011D928A95E9F7CA
:103BE000C1CF2C960FB6F894DEBF0FBECDBFDF91CC
:103BF000CF911F910895EF92FF920F931F93CF9350
:103C0000DF938C01892B09F46CC0F12CEE24E39432
:103C1000E8012196F8018491843740F4843008F05B
:103C200051C0813081F0823019F15BC0853709F4D1
:103C300044C0A8F19CE7980F903708F052C08F77E6
:103C40000E94351741C00E5F1F4FFE01C49180E2F4
:103C50008C0F883048F4C7708E2D01C0880FCA952C
:103C6000EAF70E94AB2014C08C2F0E946D162DC065
:103C70000E5F1F4FFE01C49180E28C0F883058F414
:103C8000C7708E2D01C0880FCA95EAF70E94B12037
:103C90000E94D2201AC08C2F0E94351716C00E5FCA
:103CA0001F4FFE01C491CC2381F08FE99FE0019763
:103CB000F1F700C00000C150F6CF0E5F1F4FFE01AC
:103CC000F49003C00E946D168E018F2D882309F495
:103CD0009FCFEFE9FFE03197F1F700C0000081507E
:103CE000F5CFDF91CF911F910F91FF90EF90089545
:103CF00008956093C0017093C1018093C2019093B5
:103D0000C3010C94AB1A0F931F930091C001109143
:103D1000C1012091C2013091C301DC01CB01802B94
:103D2000912BA22BB32B8093C0019093C101A09340
:103D3000C201B093C3011F910F910C94AB1A0F9362
:103D40001F930091C0011091C1012091C2013091D7
:103D5000C301DC01CB0180239123A223B3238093F1
:103D6000C0019093C101A093C201B093C3011F9100
:103D70000F910C94AB1A0F931F930091C0011091F7
:103D8000C1012091C2013091C301DC01CB01802728
:103D90009127A227B3278093C0019093C101A093DC
:103DA000C201B093C3011F910F910C94AB1A1092F2
:103DB000BC011092BD011092BE011092BF010C9483
:103DC000AB1A41E050E060E070E004C0440F551FC2
:103DD000661F771F8A95D2F74093BC015093BD01AF
:103DE0006093BE017093BF010C94AB1A41E050E0A8
:103DF00060E070E004C0440F551F661F771F8A956E
:103E0000D2F78091BC019091BD01A091BE01B0910B
:103E1000BF01482B592B6A2B7B2B4093BC0150933D
:103E2000BD016093BE017093BF010C94AB1A41E0D9
:103E300050E060E070E004C0440F551F661F771F1C
:103E40008A95D2F740955095609570958091BC0108
:103E50009091BD01A091BE01B091BF0148235923AB
:103E60006A237B234093BC015093BD016093BE0144
:103E70007093BF010C94AB1A41E050E060E070E039
:103E800004C0440F551F661F771F8A95D2F7809193
:103E9000BC019091BD01A091BE01B091BF01482726
:103EA00059276A277B274093BC015093BD0160933B
:103EB000BE017093BF010C94AB1A0F931F93009136
:103EC000BC011091BD012091BE013091BF01DC0108
:103ED000CB01802B912BA22BB32B8093BC01909311
:103EE000BD01A093BE01B093BF011F910F910C942F
:103EF000AB1A0F931F930091BC011091BD0120914B
:103F0000BE013091BF01DC01CB0180239123A223AC
:103F1000B3238093BC019093BD01A093BE01B093E5
:103F2000BF011F910F910C94AB1A0F931F93009137
:103F3000BC011091BD012091BE013091BF01DC0197
:103F4000CB0180279127A227B3278093BC019093B0
:103F5000BD01A093BE01B093BF011F910F910C94BE
:103F6000AB1A0895CF92DF92EF92FF920F931F93B7
:103F7000CF93DF938C01C090C001D090C101E0903D
:103F8000C201F090C3014091BC015091BD0160910C
:103F9000BE017091BF01C42AD52AE62AF72ACFE1D3
:103FA000D0E0D701C6010C2E04C0B695A795979511
:103FB00087950A94D2F780FF07C0B8018C2F0E9422
:103FC000DA0B8130910531F4219758F7B80180E080
:103FD0000E94DA0BDF91CF911F910F91FF90EF902C
:103FE000DF90CF90089590910C01992321F090914A
:103FF0000D01911109C020910E0130910F01F901BD
:1040000032969FEF40E030C0982F96959695969502
:104010009F30A0F4E0910E01F0910F01E90FF11D26
:10402000877021E030E0A90102C0440F551F8A9536
:10403000E2F7CA019181892B818308959091D7017C
:1040400090FF23C01F928F9387ED95E09F938F93EE
:104050000E94EB070F900F900F900F9008959F3FD5
:1040600039F04F5F4E3041F051915813F8CF0DC0E9
:104070005111F7CF942FF5CF9F3F39F0F901E90F98
:10408000F11D97FDFA9582830895089590910C0192
:10409000992321F090910D01911109C020910E01F9
:1040A00030910F01F9013296205F3F4F30C0982FB9
:1040B0009695969596959F30A8F4E0910E01F09113
:1040C0000F01E90FF11D877021E030E0A90102C066
:1040D000440F551F8A95E2F7CA0180959181892383
:1040E000818308959091D70190FF16C01F928F93FE
:1040F00089EB95E09F938F930E94EB070F900F90B1
:104100000F900F9008953196E217F30729F09081F0
:104110009813F9CF1082F7CF089581E090E0E091F5
:104120000E01F0910F01E80FF91F10820196803106
:104130009105A9F708959091D601892B8093D60116
:10414000089580959091D60189238093D601089592
:104150001092D60108959091D501892B8093D501B5
:10416000089580959091D50189238093D501089574
:104170001092D50108958093C40108951092C4014E
:10418000089580910E0190910F01FC0131969C01E0
:10419000205F3F4F80E0919191118F5FE217F3070D
:1041A000D1F70895E0910E01F0910F018091D601B1
:1041B0008083E0910E01F0910F0190818091D501F3
:1041C000892B80838091C401882361F0E0910E01E6
:1041D000F0910F019081892B80830E94C120811171
:1041E0001092C40180910E0190910F010C94EB1478
:1041F00090933B0180933A010895CF92DF92EF9222
:10420000FF926C01EE24FF24C114D104E104F104F7
:1042100021F0C701B60120E101C020E0C72ED82E51
:10422000E92EFF24C114D104E104F10419F0285F40
:10423000C701B6016B017C0154E0F694E794D79472
:10424000C7945A95D1F7C114D104E104F10419F0CF
:104250002C5FC701B6016B017C0142E0F694E79444
:10426000D794C7944A95D1F7C114D104E104F1045D
:1042700019F02E5FC701B601DC01CB01B695A795F9
:1042800097958795892B8A2B8B2B09F02F5F822F8F
:10429000FF90EF90DF90CF9008958295982F9C7CAF
:1042A000392F36953695282F237344E0249FC0017B
:1042B0001124932F982B292F2A7A2695892F8575DB
:1042C000880F822B08951F93CF93DF931F92CDB752
:1042D000DEB799830E944D21182F9981892F0E9462
:1042E0004D21212F30E0322F2227A901482BCA016E
:1042F0000F90DF91CF911F9108958091F00184304C
:1043000009F11092D80120E488E190E00FB6F8940A
:10431000A895809360000FBE2093600083B7817FD3
:10432000846083BF83B7816083BF7894889583B7A7
:104330008E7F83BF88E10FB6F8948093600010925F
:1043400060000FBE089508950895CF930E94A321A1
:104350000E947F090E94A421C0E08C2F0E94AB0A1A
:10436000811104C0CF5FCE30C1F701C081E0CF9191
:1043700008950C94BD1A82E084BD93E095BD9AEF38
:1043800097BD80936E0008952FB7F8948091D9015E
:104390009091DA01A091DB01B091DC012FBF08956B
:1043A000CF92DF92EF92FF920F931F932FB7F89463
:1043B0004091D9015091DA016091DB017091DC01EB
:1043C0002FBF6A017B01EE24FF248C0120E030E046
:1043D000C016D106E206F30610F4415051099A01C5
:1043E000281B390BC9011F910F91FF90EF90DF90AF
:1043F000CF9008951F920F920FB60F9211248F93B2
:104400009F93AF93BF938091D9019091DA01A091CE
:10441000DB01B091DC010196A11DB11D8093D90192
:104420009093DA01A093DB01B093DC01BF91AF91CF
:104430009F918F910F900FBE0F901F9018950E9423
:10444000DD11F8942FEF87EA91E6215080409040EB
:10445000E1F700C0000087E090EBDC018093F901F8
:104460009093FA01A093FB01B093FC019CE088E1DA
:104470000FB6F894A895809360000FBE90936000EB
:10448000FFCFEF92FF920F931F93CF93DF93D82F1D
:10449000C0E08C2F0E94AB0A00E010E0E82EF12C67
:1044A000C701002E02C0959587950A94E2F780FD1A
:1044B00006C00F5F1F4F0630110591F709C0602F2E
:1044C0007C2F80E00E94B80BD813F3CF81E004C0AA
:1044D000CF5FCE30F1F680E0DF91CF911F910F9149
:1044E000FF90EF900895CF93C82F8CE20E94412255
:1044F000882321F08C2FCF910C94412280E0CF9122
:104500000895CF930E94D023811102C00E94B62348
:104510008CEF95E00E945207C5E6C15049F00E9419
:104520007F098FE39CE90197F1F700C00000F5CF08
:1045300085EF95E00E94520789E20E947322811163
:1045400013C18AE20E94732281110E94B62385E082
:104550000E94732281110E941F220E94DB238093FC
:10456000D70187E00E9473228823A9F18BE10E9482
:104570007322882351F08091D70181FB222720F9F3
:1045800091E0922790FB81F90EC08EE00E94732289
:10459000882361F08091D70182FB222720F991E0E6
:1045A000922790FB82F98093D70115C080E10E9489
:1045B00073229091D701882341F093FB222720F9A1
:1045C00081E0822780FB93F904C0892F809580FBCE
:1045D00090F99093D7018091D7010E94DF230E9428
:1045E000ED238093EA0180EE0E947322882341F03C
:1045F0008091EA01982F909590FB80F98093EA01D1
:1046000089E30E947322882359F08091EA0181FB9B
:10461000222720F991E0922790FB81F98093EA010B
:1046200082EE0E947322882359F08091EA0182FB76
:10463000222720F991E0922790FB82F98093EA01EA
:1046400086EE0E947322882359F08091EA0183FB51
:10465000222720F991E0922790FB83F98093EA01C9
:1046600083EE0E947322882359F08091EA0184FB33
:10467000222720F991E0922790FB84F98093EA01A8
:1046800085E30E947322882359F08091EA0185FB1B
:10469000222720F991E0922790FB85F98093EA0187
:1046A00081E30E947322882359F08091EA0186FBFE
:1046B000222720F991E0922790FB86F98093EA0166
:1046C00081E10E947322882359F08091EA0187FBDF
:1046D000222720F991E0922790FB87F98093EA0145
:1046E0008091EA010E94F1238091EA0187FB8827EB
:1046F00080F980930D0187E20E947322C82F8EE11A
:104700000E9473228111C2608FE10E947322811185
:10471000C46080E20E9473228111C86081E20E941D
:1047200073228111C06182E20E9473228111C062F2
:1047300083E20E9473228111C06484E20E9473228A
:10474000882311F0C06802C0CC2329F08C2F0E946E
:10475000E8236C2F03C00E94E423682F70E080E000
:1047600090E0CF910C94791ECF9108956DEE7EEF7D
:1047700080E090E00E94B92D60E082E090E00E942D
:10478000AB2D60E083E090E00E94AB2D60E084E020
:1047900090E00E94AB2D60E085E090E00C94AB2DA2
:1047A00080E090E00E94A52D21E08D3E9E4F09F013
:1047B00020E0822F089582E090E00C949D2D682FD8
:1047C00082E090E00C94AB2D83E090E00C949D2D62
:1047D000682F83E090E00C94AB2D84E090E00C9483
:1047E0009D2D682F84E090E00C94AB2D8091DF012B
:1047F00080FF0BC06091130185E0689FB001112418
:1048000075956795759567952BC081FF09C0609177
:10481000130185E0689FB00111247595679520C04C
:1048200082FF07C06091130185E0689FB0011124E9
:1048300017C09091E0019923D1F060911201961771
:1048400088F72091130185E0289F90011124929F01
:10485000A001939F500D112470E0CA010E946F2D9A
:104860006038710540F46115710539F002C065E0EA
:1048700070E0862F08958FE7089581E00895809174
:10488000DF0180FF08C06091110170E075956795A8
:104890007595679521C081FF06C06091110170E098
:1048A0007595679519C082FF04C06091110170E091
:1048B00010C09091E0019923C1F06091100196170A
:1048C000A0F780911101899FC001112470E00E941E
:1048D0006F2D6038710528F46115710521F0862F60
:1048E00008958FE7089581E0089561E070E0F4CFC6
:1048F000803F21F40E94F623819504C0813F29F472
:104900000E94F6238093E3010895823F21F40E94E0
:10491000F623819504C0833F29F40E94F6238093F7
:10492000E2010895893F19F40E943F2405C08A3F9F
:1049300031F40E943F2481958093E40108958B3FD8
:1049400021F40E943F24819504C08C3F29F40E94E9
:104950003F248093E5010895843F21F48091E10193
:10496000816017C0853F21F48091E101826011C010
:10497000863F21F48091E10184600BC0873F21F4E0
:104980008091E101886005C0883F31F48091E101A8
:1049900080618093E10108958D3F21F48091DF01D2
:1049A00081600BC08E3F21F48091DF01826005C0E1
:1049B0008F3F29F48091DF0184608093DF010895A7
:1049C000803F39F48091E30187FF6CC01092E301CE
:1049D00069C0813F29F48091E3011816BCF362C0DD
:1049E0009091E201823F29F497FF5CC01092E201AE
:1049F00059C0833F19F41916CCF354C0893F41F4D0
:104A00008091E40118160CF04DC01092E4014AC0E8
:104A10008A3F29F48091E40187FF44C0F6CF8B3FA1
:104A200039F48091E50187FF3DC01092E5013AC05D
:104A30008C3F29F48091E5011816BCF333C0843F04
:104A400021F48091E1018E7F17C0853F21F4809190
:104A5000E1018D7F11C0863F21F48091E1018B7FC0
:104A60000BC0873F21F48091E101877F05C0883F1B
:104A700031F48091E1018F7E8093E10113C08D3F7D
:104A800021F48091DF018E7F0BC08E3F21F4809155
:104A9000DF018D7F05C08F3F29F48091DF018B7F7F
:104AA0008093DF018091E20181110EC08091E301CA
:104AB00081110AC08091E401811106C08091E50155
:104AC000811102C01092E00108958091D70183FF07
:104AD0007EC088E396E00E9452078091E1011F9218
:104AE0008F9383E396E09F938F930E94EB0781E37C
:104AF00096E00E9452078091E201282F332727FD7C
:104B000030953F938F938EE296E09F938F930E9410
:104B1000EB078CE296E00E9452078091E301282F78
:104B2000332727FD30953F938F9389E296E09F933B
:104B30008F930E94EB0787E296E00E9452078091D4
:104B4000E401282F332727FD30953F938F9384E28C
:104B500096E09F938F930E94EB0782E296E00E947B
:104B600052078091E501282F332727FD30953F9389
:104B70008F938FE196E09F938F930E94EB078CE1D8
:104B800096E00E9452078091E0011F928F9389E185
:104B900096E09F938F930E94EB0787E196E00E9437
:104BA00052078091DF011F928F9384E196E09F93DB
:104BB0008F930E94EB0781E196E00E9452078DB728
:104BC0009EB74C960FB6F8949EBF0FBE8DBF81EE78
:104BD00091E00E9434150E94C4219093DE018093DD
:104BE000DD0108951F93CF93DF938091DD019091B4
:104BF000DE010E94D021AC019091E001992321F0C7
:104C00002091140130E006C0209115018AE0289F10
:104C1000900111244217530708F486C08091E201E5
:104C2000C091E301D091E4011091E501811107C029
:104C3000C11176C0D11174C0111172C075C09F3FEF
:104C400019F09F5F9093E001181624F40E94F62358
:104C50008093E2018091E20187FF05C00E94F62364
:104C600081958093E2011C1624F40E94F623809320
:104C7000E3018091E30187FF05C00E94F62381953F
:104C80008093E3016091E201662339F1C091E30171
:104C9000CC2319F1772767FD7095872F972F0E94F6
:104CA000742C23E333E343E35FE30E94D82C0E9498
:104CB000412C6093E2016C2F772767FD7095872F59
:104CC000972F0E94742C23E333E343E35FE30E94B6
:104CD000D82C0E94412C6093E3011D1624F40E94FD
:104CE0003F248093E4018091E40187FF05C00E9486
:104CF0003F2481958093E401111624F40E943F24FF
:104D00008093E5018091E50187FF05C00E943F2463
:104D100081958093E501DF91CF911F910C946525DA
:104D20009F3F09F08ECF96CFDF91CF911F910895CD
:104D3000E1EEF1E085E0DF011D928A95E9F710923E
:104D4000E0011092DF0108958BE598E00E94520780
:104D50001F9281E08F931F9285E08F938DE098E002
:104D60009F938F930E94EB070F900F900F900F90DF
:104D70000F900F9008958330E9F128F4813061F0AD
:104D8000823009F10895853009F462C008F449C001
:104D9000863009F474C0089580911501262F30E003
:104DA000280F311D2F3F310524F4680F6093150142
:104DB00003C08FEF80931501809115011F928F938F
:104DC00086E497E072C080911401262F30E0280F0E
:104DD000311D2F3F310524F4680F6093140103C087
:104DE0008FEF80931401809114011F928F9384E3BD
:104DF00097E05BC080911301262F30E0280F311D12
:104E00002F3F310524F4680F6093130103C08FEF27
:104E100080931301809113011F928F9381E297E099
:104E200044C080911201262F30E0280F311D2F3F02
:104E3000310524F4680F6093120103C08FEF809353
:104E40001201809112011F928F938CE097E02DC088
:104E500080911101262F30E0280F311D2F3F3105A1
:104E600024F4680F6093110103C08FEF8093110148
:104E7000809111011F928F9383EF96E016C080916D
:104E80001001262F30E0280F311D2F3F310524F46B
:104E9000680F6093100103C08FEF80931001809121
:104EA00010011F928F9388ED96E09F938F930E943D
:104EB000EB070F900F900F900F900895833081F1C2
:104EC00028F4813059F08230D1F00895853009F40A
:104ED00049C0B8F1863009F456C008958091150193
:104EE000681720F4861B8093150102C010921501EB
:104EF000809115011F928F9389EC96E054C08091A8
:104F00001401681720F4861B8093140102C01092CC
:104F10001401809114011F928F9387EB96E043C098
:104F200080911301681720F4861B8093130102C03F
:104F300010921301809113011F928F9384EA96E0DF
:104F400032C080911201681720F4861B80931201F1
:104F500002C010921201809112011F928F938FE86C
:104F600096E021C080911101681720F4861B809380
:104F7000110102C010921101809111011F928F93B3
:104F800086E796E010C080911001681720F4861B18
:104F90008093100102C010921001809110011F92A5
:104FA0008F938BE596E09F938F930E94EB070F9072
:104FB0000F900F900F900895CF93C82F1F928F934B
:104FC00080E699E09F938F930E94EB0781E090E049
:104FD000A0E0B0E0BC01CD0104C0660F771F881FC0
:104FE000991FCA95D2F70E94791E0F900F900F90CB
:104FF0000F90CF910C94BD1ACF938D3109F465C0F9
:10500000B0F58E3009F4CCC100F5873009F49BC1AE
:10501000A8F4863009F06DC28091D701817F8E7F20
:105020008093D70185E699E00E94520781EA9DE0CE
:105030000E94520781E08093E70180C1883009F423
:105040004FC08B3009F47CC154C2863109F4F0C1E1
:1050500038F4803109F4B8C1813109F430C249C251
:10506000893109F4CEC18B3109F486C142C285333E
:1050700009F437C248F4873209F433C208F433C262
:10508000893209F42EC235C2833438F48A3308F0E9
:105090002CC2883309F454C12CC2833409F421C2D0
:1050A000883409F026C20E94BD1A80E99DE00E9462
:1050B00052079FEF23ED80E3915020408040E1F7BD
:1050C00000C000000E941F2239C180EB9DE00E94B9
:1050D00052070E94FB2B0E94DF140E94110D2EC16B
:1050E00085EA9DE00E94520786E79BE00E945207F6
:1050F0000E94E4231F928F9383E79BE09F938F93FB
:105100000E94EB0781E79BE00E9452070E94DB238D
:10511000C82F8EE59BE00E9452071F92CF9389E52E
:105120009BE09F938F930E94EB0787E59BE00E9493
:1051300052078DE49BE00E9452078C2F81701F92D2
:105140008F938AE49BE09F938F930E94EB0788E400
:105150009BE00E9452078EE39BE00E945207C1FB36
:10516000882780F91F928F938BE39BE09F938F9307
:105170000E94EB0789E39BE00E9452078DE29BE0CF
:105180000E945207C2FB882780F91F928F938AE200
:105190009BE09F938F930E94EB0788E29BE00E9425
:1051A00052078FE19BE00E945207C3FBCC27C0F956
:1051B0001F92CF938CE19BE09F938F930E94EB070C
:1051C0008AE19BE00E9452070E94ED23C82F86E0EF
:1051D0009BE00E9452071F92CF9381E09BE09F9338
:1051E0008F930E94EB078FEF9AE00E94520786EEA2
:1051F0009AE00E9452078C2F81701F928F9383EE4A
:105200009AE09F938F930E94EB078DB79EB780968D
:105210000FB6F8949EBF0FBE8DBF81EE9AE00E943C
:1052200052078AEC9AE00E945207C1FB882780F956
:105230001F928F9387EC9AE09F938F930E94EB07C6
:1052400085EC9AE00E94520783EB9AE00E94520795
:10525000C2FB882780F91F928F9380EB9AE09F937F
:105260008F930E94EB078EEA9AE00E9452078CE926
:105270009AE00E945207C3FB882780F91F928F9300
:1052800089E99AE09F938F930E94EB0787E99AE060
:105290000E9452078DE89AE00E945207C4FB8827BB
:1052A00080F91F928F938AE89AE09F938F930E94D0
:1052B000EB0788E89AE00E94520786E79AE00E948E
:1052C0005207C5FB882780F91F928F9383E79AE0E6
:1052D0009F938F930E94EB0781E79AE00E94520709
:1052E00085E59AE00E945207C6FB882780F91F9245
:1052F0008F9382E59AE09F938F930E94EB0780E55E
:105300009AE00E94520788E49AE00E945207C7FB85
:10531000CC27C0F91F92CF9385E49AE09F938F9397
:105320000E94EB0783E49AE00E9452078DB79EB774
:105330004C960FB6F8949EBF0FBE8DBFC1E0DEC085
:105340008CE899E05BC08091D701C82FC17080FFC5
:1053500009C083E89DE00E9452078091D701817FB8
:105360008E7F47C087E79DE00E9452078091D7015A
:1053700081608093D701E2CF9091D70191FBCC2738
:10538000C0F981E0C827892FC0FB81F98093D7013C
:10539000CC2319F08AE69DE027C08CE59DE02EC065
:1053A0009091D70192FBCC27C0F981E0C827892FC3
:1053B000C0FB82F98093D701CC2319F08DE49DE0E6
:1053C00013C08DE39DE01AC09091D70193FBCC27C9
:1053D000C0F981E0C827892FC0FB83F98093D701EA
:1053E000CC2351F081E39DE00E9452078091D701C8
:1053F00081608093D70182C084E29DE00E945207C1
:105400009DCF85E19DE00E94520789EE9CE00E94BD
:1054100052078CEA9CE00E94520785E89CE00E94BB
:10542000520781E49CE00E94520786E19CE0E6CFAF
:1054300088E09CE00E9452070E94DF141F928F9325
:105440008EEE9BE09F938F930E94EB0780910C015F
:105450001F928F9387ED9BE09F938F930E94EB07A2
:1054600080916E011F928F9384EC9BE09F938F93AA
:105470000E94EB0780910D011F928F9381EB9BE0BF
:105480009F938F930E94EB078091D9019091DA014D
:10549000A091DB01B091DC01BF93AF939F938F93F9
:1054A0008DE99BE09F938F930E94EB078DB79EB78A
:1054B00046960FB6F8949EBF0FBE8DBF3FCF0E9499
:1054C000BD1AC0910D0181E0C827C0930D01CC2306
:1054D00029F083E99BE00E94520710C088E89BE016
:1054E0008DCF80E003C08D5101C089530E94DC271D
:1054F00025CF86E89BE00E945207C0E08C2FCF9119
:10550000089580E0089580E00895CF93C82F80919A
:10551000E701813081F020F0823009F44FC045C1AD
:10552000E0910E01F0910F018081813169F08232AA
:1055300009F03DC109C0E0910E01F0910F01808199
:10554000813111F0823261F48C2F0E94812A811105
:1055500004C08C2F0E94FC272FC081E090E02CC05B
:105560008C2F0E94832A811126C0C431E1F070F48F
:10557000CB3081F0C031D1F40E94A42688E599E0B7
:105580000E94520782E08093E70115C0C93259F0AA
:10559000C83361F485E699E00E9452078CE599E0F2
:1055A0000E94520708C01092E70103C186E599E006
:1055B0000E945207FEC081E08170FDC0C43220F518
:1055C000CE3108F0C0C0CB3099F1C8F4C73009F033
:1055D000D2C08AE08093150194E19093140193E086
:1055E000909313018093120188E08093110188E267
:1055F000809310018CEF97E00E945207BFC0C33127
:1056000049F1C431C1F0B7C0CB3409F4A9C028F4C2
:10561000C93289F0C83361F0AEC0C13509F49EC00B
:10562000C23509F499C0CE3409F0A5C06AE09EC025
:105630000E94A426A3C08091E601882319F010924D
:10564000E6019CC089E098E00E94520781E08093C7
:10565000E701B1C083EE97E00E94520781ED97E029
:105660000E945207809115011F928F938EEC97E054
:105670009F938F930E94EB078CEC97E00E94520758
:105680008AEB97E00E945207809114011F928F933A
:1056900087EB97E09F938F930E94EB0785EB97E052
:1056A0000E94520786EA97E00E94520780911301F8
:1056B0001F928F9383EA97E09F938F930E94EB074B
:1056C00081EA97E00E94520780E997E00E94520722
:1056D000809112011F928F938DE897E09F938F9393
:1056E0000E94EB078BE897E00E94520786E797E05D
:1056F0000E945207809111011F928F9383E797E0D8
:105700009F938F930E94EB0781E797E00E945207D7
:105710008AE597E00E945207809110011F928F93B3
:1057200087E597E09F938F930E94EB0785E597E0CD
:105730000E9452078DB79EB748960FB6F8949EBF49
:105740000FBE8DBF1BC0CE51EC2FF0E0E15DFE4FD0
:1057500080818093E60112C061E003C061E006C071
:105760006AE08091E6010E94BB2608C08091E601B4
:105770000E945E2703C08AEF97E013C08091E60184
:10578000882369F01F928F9384EF97E09F938F9304
:105790000E94EB070F900F900F900F9004C081EFC5
:1057A00097E00E94520781E006C01092E70180E076
:1057B00002C080E001CFCF910895E1E8F0E0808160
:1057C000886080838081816080838FB7F89493E0C4
:1057D0009093890090ED909388008FBF0895EFE635
:1057E000F0E08081826080830895EFE6F0E08081C0
:1057F0008D7F80830895EFE6F0E0908182E0892735
:10580000808308951F920F920FB60F9211242F9349
:105810003F934F935F936F937F938F939F93AF9338
:10582000BF93EF93FF938091E8019091E901019676
:105830009093E9018093E801811103C082E00E9406
:10584000110DE091E901E695E695F0E0E054F24FA4
:10585000E4918091E8018E1303C080E00E94110D55
:10586000FF91EF91BF91AF919F918F917F916F9138
:105870005F914F913F912F910F900FBE0F901F900E
:10588000189504D06894B1118DC0089570D088F037
:105890009F5790F0B92F9927B751A0F0D1F0660F1C
:1058A000771F881F991F1AF0BA95C9F712C0B13037
:1058B00081F077D0B1E0089574C0672F782F8827E2
:1058C000B85F39F0B93FCCF3869577956795B39576
:1058D000D9F73EF490958095709561957F4F8F4FE5
:1058E0009F4F0895E89409C097FB3EF490958095EA
:1058F000709561957F4F8F4F9F4F9923A9F0F92F96
:1059000096E9BB279395F695879577956795B79513
:10591000F111F8CFFAF4BB0F11F460FF1BC06F5FF9
:105920007F4F8F4F9F4F16C0882311F096E911C00B
:10593000772321F09EE8872F762F05C0662371F02C
:1059400096E8862F70E060E02AF09A95660F771F40
:10595000881FDAF7880F9695879597F9089557FD70
:105960009058440F551F59F05F3F71F04795880FCD
:1059700097FB991F61F09F3F79F087950895121664
:1059800013061406551FF2CF4695F1DF08C0161610
:1059900017061806991FF1CF8695710561050894C1
:1059A0000895E894BB2766277727CB0197F90895D8
:1059B0000BD078C069D028F06ED018F0952309F08C
:1059C0005AC05FC01124EECFCADFA0F3959FD1F378
:1059D000950F50E0551F629FF001729FBB27F00D9D
:1059E000B11D639FAA27F00DB11DAA1F649F6627F2
:1059F000B00DA11D661F829F2227B00DA11D621F41
:105A0000739FB00DA11D621F839FA00D611D221FFA
:105A1000749F3327A00D611D231F849F600D211DDE
:105A2000822F762F6A2F11249F5750408AF0E1F081
:105A300088234AF0EE0FFF1FBB1F661F771F881FCA
:105A400091505040A9F79E3F510570F014C0AACF65
:105A50005F3FECF3983EDCF3869577956795B795B5
:105A6000F795E7959F5FC1F7FE2B880F911D9695DF
:105A7000879597F9089597F99F6780E870E060E04F
:105A800008959FEF80EC089500240A9416161706D7
:105A900018060906089500240A941216130614061F
:105AA00005060895092E0394000C11F4882352F082
:105AB000BB0F40F4BF2B11F460FF04C06F5F7F4F3A
:105AC0008F4F9F4F0895991B79E004C0991F961737
:105AD00008F0961B881F7A95C9F78095089597FB63
:105AE000072E16F4009407D077FD09D00E94892D67
:105AF00007FC05D03EF4909581959F4F08957095D1
:105B000061957F4F0895EE0FFF1F0590F491E02DF2
:105B10000994AA1BBB1B51E107C0AA1FBB1FA617F4
:105B2000B70710F0A61BB70B881F991F5A95A9F746
:105B300080959095BC01CD010895F999FECF92BD55
:105B400081BDF89A992780B50895A8E1B0E042E0B8
:105B500050E00C94C02D262FF999FECF1FBA92BDAC
:105B600081BD20BD0FB6F894FA9AF99A0FBE01963E
:105B700008950E94AB2D272F0C94AC2DDC01CB0196
:105B8000FC01F999FECF06C0F2BDE1BDF89A31964D
:105B900000B40D9241505040B8F70895F894FFCFEB
:105BA0002002120D030EE00DAC0D780D0101C501B0
:105BB00028080A03140A3F4D3620394605F904C364
:105BC00004A3046A04DD03F6030F04280448040157
:0A5BD000020304050607080900009F
:00000001FF
